:10000000B2017C290408A70006108610861083160A
:10001000061086108610870183122708B2182B2835
:100020003A30A100FC3047213330A6003E2010308A
:10003000A100683047213E20643046213E20383000
:100040002A200C302A2001302A2006302A20B2141F
:1000500027082B283214A600321C39288610033CAE
:10006000031C3E283E201330A10088304721031492
:1000700008003214FE3C031977298614061426085A
:100080008700000032100610C83046210314080013
:10009000003803197729A800200884002118831745
:1000A000A001A101A81B5C280008A000A81C7729BA
:1000B000840A0008A10077292C210005031DA00A4D
:1000C00077296400772003186128EA20A801083006
:1000D000A300EB2077200318A80AAB1EA801A20CEE
:1000E000A30B6928AB1AA213EB20220808003608DC
:1000F0008400340884178004841300052B1B340605
:10010000FF3E0800A401A501B3127221D33E0319DA
:10011000B3162D3EC63E031885280A3E031C8528CB
:10012000A2000310240DA000250DA100200DA10D9B
:10013000A4070318A10A2108A507A40DA50D2208EC
:10014000A4070318A50AA9030319AD287221C63E06
:100150000318AD280A3E03189028B31EB428A4093A
:10016000A509A40A0319A50A24087729A6003608B8
:1001700084008030B3050830A70003100318B30AC9
:10018000D020A60CA70BBE280000AB1A330CD02041
:100190007A210314D0202F08A3002E083A217729B2
:1001A0008413AB1FDF28000834042B1F34068000A3
:1001B000841700083404031C34068000EB28000870
:1001C0003404031C34062B1B3406800084173409C6
:1001D0008005EB2833172B081F39003EA1002A08A1
:1001E0000E3E0318A10A331F47293313A000031042
:1001F000A10CA00C0310A10C200C4729B313290853
:100200000319B3170530A8002730A30010301421BC
:100210000330A300E8301421A30164301421A301AA
:100220000A30142124081B29A2002508A100240853
:10023000A00056212008A000A8030319B313290821
:10024000031925292802031808002008031DB313E9
:10025000B31B0800303E722901308A002808073994
:10026000820701340234043408341034203440341A
:100270008034A301A200FF30A207031CA307031CC4
:1002800077290330A100E63047213B29A101FC3E3C
:10029000A000A109031C5229FF300000A007031889
:1002A0004D29A0076400A10F4C290800A501A40155
:1002B0001030A600210DA40DA50D2208A4022308CC
:1002C000031C230FA50203186C292208A407230886
:1002D0000318230FA5070310A00DA10DA60B5A2983
:1002E00020087729840031088A00300882008313AF
:1002F0000313831264000800831607309F008312E3
:10030000C401051483160510831285148316851005
:100310008312851583168511831206118316061123
:10032000051485148515061583128512831685120A
:1003300083120130A300F4303A218516831685120A
:1003400083120130A300F4303A2164000518AA2971
:100350004410AB29441464008518B029C410B12995
:10036000C41464008519B6294411B72944156400E2
:1003700004304402031CC1290430C4025430C600B6
:10038000C3294E30C6004408A200033C031CE829E0
:100390000310220DA207D821A000A20AD821A10093
:1003A000A20AD82148202008C0002108C100E8295D
:1003B00001308A00220882072034003400342D34B2
:1003C000033400348C3401340034543400340034A9
:1003D0004408A200033C031C0D2A0310220DA207AF
:1003E000FD21A000A20AFD21A100A20AFD214820B2
:1003F0002008C2002108C3000D2A02308A0022080A
:10040000820700344B340034B03404340034603498
:1004100009340034803425340034640046084E3CEE
:10042000031D132A4117831606158611C83083123F
:1004300039210630B6000830B4004008AA0041084F
:10044000AB00AE01AF014330B6204C30B620433094
:10045000B6204430B6202030B6205030B62072305E
:10046000B6206F30B6206730B6207230B6206130CB
:10047000B6206D30B6202030B6207630B620313030
:10048000B6202E30B6203130B6200D30B6200A30DE
:10049000B62010242030CA000630B6000430B40064
:1004A0004008AA004108AB0061200D3C031D542AFE
:1004B0006120CC000630B6000830B4004008AA0025
:1004C0004108AB00AE01AF015330B6207430B62006
:1004D0006130B6207230B6207430B6206930B62054
:1004E0006E30B6206730B6200D30B6200A30B62008
:1004F0000630B6000430B4004008AA004108AB0042
:100500006120CA000630B6000830B4004008AA00D6
:100510004108AB00AE01AF014A08B6200D30B6204D
:100520000A30B62064004A085C3C031D982ACE2A93
:1005300064004A085D3C031D9E2A162B64004A088D
:100540005B3C031DA42A282B64004A08083C031DB9
:10055000B42AFE3003201030032020300320FE3068
:10056000032010300320CD2A64004A08093C031DF3
:10057000C52A0130C9006400063049020318C42AA4
:1005800020300320C90FBB2ACD2A64004A080D3C45
:10059000031DCB2ACD2A4A080320782A0630B6004C
:1005A0000430B4004008AA004108AB000330A900A1
:1005B0006130B000B1018220CB0064004B08013CE7
:1005C000031DE92AFE300320013003201E303921AB
:1005D000152B64004B08803C031DF32AFE300320DA
:1005E00080300320152B64004B08C03C031DFD2AFE
:1005F000FE300320C0300320152B64004B08943CD0
:10060000031D072BFE30032094300320152B6400BC
:100610004B08D43C031D112BFE300320D4300320A3
:10062000152BFE3003204B080320782A0630B60035
:100630000430B4004008AA004108AB000330A90010
:100640006130B000B1018220CB004B080320782A32
:100650000630B6000430B4004008AA004108AB00E0
:100660000230A9006130B000B1018220CB006400EB
:100670004B081E3C031D412B8611831686118312E5
:10068000062C64004B081F3C031D4B2B861583165C
:1006900086118312062C64004B08283C031D552B41
:1006A0000612831606128312062C64004B08293C9E
:1006B000031D5F2B0616831606128312062C640098
:1006C0004B08323C031D692B861283168612831257
:1006D000062C64004B08333C031D732B86168316CF
:1006E00086128312062C64004B083C3C031D7D2BB4
:1006F0000613831606138312062C64004B083D3C38
:10070000031D872B0617831606138312062C64001D
:100710004B08463C031D912B8613831686138312C8
:10072000062C64004B08473C031D9B2B8617831641
:1007300086138312062C64004B08623C031D002CB8
:100740000630B6000430B4004008AA004108AB00EF
:100750000330A9006130B000B1018220C500023031
:10076000A9006130B000B1018220B8000230A900B8
:100770006130B000B1018220B9000230A9006130BF
:10078000B000B1018220BA000230A9006130B0008F
:10079000B1018220BB000230A9006130B000B1017C
:1007A0008220BC000230A9006130B000B10182207B
:1007B000BD000230A9006130B000B1018220BE004E
:1007C0000230A9006130B000B1018220BF00FE30CC
:1007D00003204508032038080320390803203A087D
:1007E00003203B0803203C0803203D0803203E086B
:1007F00003203F080320FE30032080300320062C16
:1008000064004B08633C031D062CD924782A63003E
:10081000072CFE300320013003201E303921080050
:10082000851683168512870183120130A3002C30B0
:100830003A21FE30032040300320003003200430F2
:100840000320023003201F30032002300320043035
:1008500003200030032000300320FE3003208030CE
:100860000320FE30032048300320003003200430F2
:100870000320083003201F300320083003200430F9
:1008800003200030032000300320FE30032080309E
:100890000320FE30032050300320003003200430BA
:1008A00003200E30032015300320043003200430D1
:1008B00003200030032000300320FE30032080306E
:1008C0000320FE3003205830032000300320003086
:1008D00003200430032004300320153003200E30A1
:1008E00003200430032000300320FE30032080303A
:1008F0000320FE300320603003201F30032011301E
:100900000320113003201130032011300320113057
:100910000320113003201F300320FE3003208030DD
:100920000320FE30032068300320043003200E3003
:1009300003201F30032000300320003003201F302D
:1009400003200E30032004300320FE3003208030CB
:100950000320FE30032070300320023003200630D5
:1009600003200E3003201E3003200E3003200630FB
:1009700003200230032000300320FE3003208030AB
:100980000320FE30032078300320083003200C3091
:1009900003200E3003200F3003200E3003200C30D4
:1009A00003200830032000300320FE300320803075
:1009B0000320FE3003200130032032303921FE3085
:1009C0000320803003205330032065300320723031
:1009D000032069300320613003206C300320203075
:1009E0000320433003204C300320433003204430A5
:1009F00003202030032076300320313003202E30B6
:100A0000032031300320FE300320C0300320423069
:100A100003206130032075300320643003203A3016
:100A200003202030032046080320A9014208A40027
:100A30004308A5000230B000B101FE20FE300320C3
:060A400002300320080053
:02400E00323F3F
:00000001FF
